:1000000084C09FC09EC09DC084C297C255C26BC2AF
:1000100098C097C096C095C094C0B5C2B7C2B9C2C7
:10002000BBC2BDC2BFC2C1C2C3C21CC31EC320C3A8
:1000300027C32EC330C337C33EC345C34CC354C3C9
:100040005BC362C369C370C377C396C3ACC3ABC39E
:10005000AAC3A9C394C3A7C3A6C3A5C3A4C391C37A
:10006000A2C3A1C3A0C39FC38EC39DC39CC39BC394
:100070009AC399C398C397C396C395C394C393C3B4
:1000800092C391C390C38FC38EC38DC38CC38BC3E4
:100090008AC389C388C387C386C385C384C383C314
:1000A00082C381C380C37FC37EC37DC37CC36EC351
:1000B0007AC379C378C377C376C375C374C373C374
:1000C00072C367C370C36FC36EC36DC364C36BC3B6
:1000D0006AC369C368C362C366C365C364C363C3D9
:1000E0005FC361C360C35FC35EC35DC35CC35BC307
:1000F0005AC359C358C357C356C355C354C353C334
:1001000052C351C350C34FC34DC311241FBE20E07F
:10011000A89521BD20E025BFE4E4F9E0A0E6B0E029
:1001200020E003C0C89531960D92A036B207D1F7F2
:10013000A0E6B0E020E001C01D92AC37B207E1F7C5
:10014000E8C300C018958FEF8ABB17BA81E484BB5F
:100150008FEF88BB8EEF85BBAE9880E48BBB089594
:1001600010926D00109274001092680084E18093E8
:10017000650010927A00109269008FEF80937900E9
:100180001092610010926E001092700010926F0039
:1001900010926C0010926B001092730082E390E05A
:1001A000909363008093620010927200109271002D
:1001B00021E020936A001092640085E5809360003E
:1001C00083EE9AED909378008093770087E49BED1F
:1001D00090937600809375008BE99FEF9093670072
:1001E0008093660086B388231CF420937A00E3D1C1
:1001F000089580E18AB98FEC89B9089580EA8FBDAE
:100200001EBC0895FBDF08958BB1992787FD90955B
:100210008827990F881F9927089595DFA1DFF2DFBE
:10022000E8DF08951092730099278230910509F450
:100230006DC08330910554F5009711F0019749F096
:100240001EBC10926E001092610010926D008FEF34
:100250007AC010926A0081E080936D0080E88093FC
:10026000610080E180936E0080916600909167004C
:100270009093700080936F0080917500909176004C
:1002800090936C0080936B008FE65DC08330910586
:1002900001F10497A9F681E080936A0084E08093DD
:1002A0006D0080E28093610080E180936E00809118
:1002B0007500909176009093700080936F0080910C
:1002C00066009091670090936C0080936B008FECB8
:1002D0003AC010926A0083E080936D0080E28093C0
:1002E000610080E480936E008091660090916700C9
:1002F0009093700080936F008091750090917600CC
:1003000090936C0080936B008FE91DC081E0809317
:100310006A0082E080936D0080E88093610080E451
:1003200080936E008091750090917600909370009C
:1003300080936F00809166009091670090936C00AD
:1003400080936B008FE380937900089580916D0016
:10035000992782309105E9F0833091057CF400976C
:1003600011F0019741F01EBC10926E0010926100D6
:1003700010926D0010C0DF9ADC980DC0833091059B
:1003800029F0049781F7DC9ADD9805C0DD9ADE98A4
:1003900002C0DE9ADF981EBC8FEF80937900109226
:1003A0006E001092610010926D000895909173009C
:1003B00080917100980F90937300943618F480E048
:1003C00090E005C094569093730081E090E008950A
:1003D00080916D00882309F46EC080916A0081309D
:1003E00089F180916B0090916C00209162003091B6
:1003F0006300820F931F90936C0080936B00809139
:100400006F0090917000821B930B9093700080930B
:100410006F00CCDF892B49F080916B0090916C00CC
:10042000019690936C0080936B0020916B0030914B
:100430006C00809166009091670082179307D8F551
:1004400085DF39C080916F0090917000209162002B
:1004500030916300820F931F9093700080936F0020
:1004600080916B0090916C00821B930B90936C00B9
:1004700080936B009BDF892B91F080916F009091AE
:10048000700001969093700080936F0080916B00D4
:1004900090916C00019790936C0080936B00209179
:1004A0006F00309170008091660090916700821714
:1004B000930708F44BDF08951F920F920FB60F9227
:1004C00011248F939F9389B39091790089238BBBDB
:1004D00081E080936400A8989F918F910F900FBE48
:1004E0000F901F9018951F920F920FB60F92112424
:1004F0008F9383B382FF03C08B7F85BB02C0846070
:1005000085BB81EB82BF8F910F900FBE0F901F9024
:1005100018951F920F920FB60F9211248F939F93ED
:1005200089B390916100892B8BBBA89A9F918F9181
:100530000F900FBE0F901F9018951F920F920FB63D
:100540000F9211248F939F9389B390916E00892B02
:100550008BBB9F918F910F900FBE0F901F9018959E
:1005600053DE892B39F18CB1282F2F7082958F7033
:100570009927AA27BB27F92FE82FE830F105D0F4F7
:10058000E35FFF4F0994822F37D014C0822F48D0E9
:1005900011C0822F5BD00EC081E044DE0BC082E030
:1005A00041DE08C083E03EDE05C084E03BDE02C0E1
:1005B000822FCCD0089586B320E080FF06C02F5F45
:1005C0008695273010F480FDFACF283008F020E01F
:1005D000822F9927880F991F8E5F80937B00822F2F
:1005E00035D0089583B385FD06C099B38FEF8BBBDB
:1005F0009D9BFECF9BBB0895982F80916900981713
:1006000011F410927A0089B321E030E002C0220F89
:10061000331F9A95E2F7922F909589238BBB08950B
:10062000382F383090F480916900381759F029B389
:1006300081E090E002C0880F991F3A95E2F7282BDD
:100640002BBB03C010927A00F2CF08959927AA27F6
:10065000BB27F92FE82FE031F10508F076C0EB5EFB
:10066000FF4F099482E390E038C089E190E035C003
:1006700080E190E0909363008093620083E463C024
:100680008CE090E0909363008093620082E35BC013
:100690008AE090E022C088E090E09093630080932D
:1006A000620081E250C087E090E090936300809305
:1006B00062008EE048C086E090E0909363008093F3
:1006C000620089E140C085E090E0909363008093F0
:1006D000620088E338C085E090E0909363008093E7
:1006E00062001092730031C084E090E09093630048
:1006F0008093620087E327C084E090E090936300DA
:100700008093620081E11FC083E090E090936300DA
:100710008093620085E517C083E090E090936300CA
:100720008093620089E30FC083E090E090936300C0
:100730008093620081E207C083E090E090936300C1
:10074000809362008DE0809373000895982F983015
:1007500028F481E080937A00909369000895809155
:1007600065009927AA27BB27F92FE82FE036F10566
:10077000D0F4EB5DFF4F099481E054DD14C0DA98AA
:1007800012C0DB9810C082E04DDD0DC083E04ADD71
:100790000AC0D99A08C084E045DD05C0DA9A03C0D2
:1007A000DB9A01C0D998089590E083B382FF02C01C
:1007B00090E001C09F5F9A30C0F3089520E083B3BA
:1007C000982F947082FF02C02F5F01C0292F2A301A
:1007D000B0F3089586B3882304F5809174008F5F89
:1007E0008093740090917B008917C0F01092740080
:1007F000809168008F5F80936800843178F0109258
:100800006800809165008F5F80936500843611F0E9
:10081000A6DF04C010926500FBCFA2DED9DD0895EB
:1008200080916D008823B1F01092640080916F0078
:10083000909170009BBD8ABD80916B0090916C007F
:1008400099BD88BD80917700909178009DBD8CBD49
:1008500082E08EBD089580916D00882321F0809103
:100860006400882349F01EBC10926400B3DF86B395
:1008700088233CF4A0DE05C080916400813079F7C4
:10088000F2CF089590E0292F80FF01C09F5F8695E9
:100890002F5F2830C8F39170892F99270895809190
:1008A0007A008823A9F180916000882369F1809102
:1008B0006000887BE7DF482F3091600030FF16C072
:1008C00029B381E090E00090690002C0880F991F71
:1008D0000A94E2F7282B2BBB832F86958093600028
:1008E0004423B1F080688093600012C029B381E096
:1008F00090E00090690002C0880F991F0A94E2F707
:10090000809528232BBBE8CF8FEF80936000CFCF5B
:100910000895CFE5D2E0DEBFCDBF7FDC80EE89BF9A
:10092000789442DFC0E05EDEC13021F047DFC1E0F5
:10093000AE9803C039DFC0E0AE9A72DF8CDFAFDF64
:04094000F2CFFFCF24
:00000001FF
